:020000040800F2
:1000000010DC012029020008AD280008D1230008D7
:10001000A92800085D05000829300008000000003C
:10002000000000000000000000000000512900084E
:100030007906000800000000E1280008B529000842
:10004000430200084302000843020008430200087C
:1000500043020008430200087D060008430200082E
:1000600043020008890600089506000843020008BC
:10007000BD050008430200084302000843020008CF
:10008000430200084302000843020008430200083C
:10009000610500087105000843020008A106000878
:1000A000430200084302000843020008430200081C
:1000B000430200084302000843020008430200080C
:1000C00043020008430200084302000843020008FC
:1000D00043020008F92F000843020008113000080D
:1000E00043020008430200084302000843020008DC
:1000F00043020008430200084302000843020008CC
:1001000043020008430200084302000843020008BB
:1001100043020008430200084302000843020008AB
:100120004302000843020008CD050008DD05000871
:10013000430200084302000843020008430200088B
:1001400081050008910500084302000843020008E9
:10015000430200084302000843020008430200086B
:10016000430200084302000843020008430200085B
:100170004302000843020008430200080000000098
:10018000430200084302000800F002F800F03CF8C7
:100190000AA090E8000C82448344AAF10107DA45E2
:1001A00001D100F031F8AFF2090EBAE80F0013F0F8
:1001B000010F18BFFB1A43F0010318473C4D000024
:1001C0007C4D0000103A24BF78C878C1FAD8520795
:1001D00024BF30C830C144BF04680C6070470000C1
:1001E0000023002400250026103A28BF78C1FBD840
:1001F000520728BF30C148BF0B6070471FB504F0DD
:1002000049FE1FBD10B510BD00F054F91146FFF7AF
:10021000F5FF02F04DFF00F072F903B4FFF7F2FFB3
:1002200003BC00F075F90000094880470948004701
:10023000FEE7FEE7FEE7FEE7FEE7FEE7FEE7FEE796
:10024000FEE7FEE704480549054A064B70470000F3
:100250006D2A00088901000810D0012010DC01205F
:1002600010D4012010D4012053EA020C00F0698060
:100270002DE9F04B4FF00006002B1FBFB3FA83F5BA
:1002800003FA05F424FA05F65E4012BF1643B2FAEB
:1002900082F502FA05F4C5F120051EBF22FA05FC1D
:1002A00044EA0C04203556EA044C4FEA144418BFC3
:1002B000641C4FF000084FF00009904271EB030CF2
:1002C00039D3002919BFB1FA81F701FA07F6B0FA5C
:1002D00080F700FA07F6C7F120071EBF20FA07FCD7
:1002E00046EA0C062037B6FBF4FCA7EB0507103FE7
:1002F00007F01F0BCBF120062CFA06F60CFA0BFBCD
:1003000044BFB3460026202FA4BF5E464FF0000B2B
:100310005BEA060C08BF4FF0010B19EB0B0948EB29
:100320000608ABFB027C06FB02CC0BFB03CCC01B1C
:1003300071EB0C01C1E70B46024641464846BDE859
:10034000F08B13B5084318BF4FF0FF300146AFF3F1
:100350000080BDE81C407047032A40F2308010F056
:10036000030C00F0158011F8013BBCF1020F624450
:1003700098BF11F801CB00F8013B38BF11F8013BE1
:10038000A2F1040298BF00F801CB38BF00F8013B8E
:1003900011F0030300F02580083AC0F0088051F8FE
:1003A000043B083A51F804CBA0E80810F5E7121D09
:1003B0005CBF51F8043B40F8043BAFF30080D20728
:1003C00024BF11F8013B11F801CB48BF11F8012BF4
:1003D00024BF00F8013B00F801CB48BF00F8012B17
:1003E000704710B5203AC0F00B80B1E81850A0E873
:1003F0001850B1E81850A0E81850203ABFF4F5AFF3
:100400005FEA027C24BFB1E81850A0E8185044BF4E
:1004100018C918C0BDE810405FEA827C24BF51F8BB
:10042000043B40F8043B08BF7047D20728BF31F8AF
:10043000023B48BF11F8012B28BF20F8023B48BF00
:1004400000F8012B704702F0FF0343EA032242EA5F
:10045000024200F002B84FF0000200B51346944685
:100460009646203922BFA0E80C50A0E80C50B1F10C
:100470002001BFF4F7AF090728BFA0E80C5048BF20
:100480000CC05DF804EB890028BF40F8042B08BFBE
:10049000704748BF20F8022B11F0804F18BF00F8BA
:1004A000012B704770477047704700000048704745
:1004B00010C001207546FFF7F9FFAE4605006946FA
:1004C000534620F00700854618B020B5FFF7BAFE66
:1004D000BDE820404FF000064FF000074FF0000845
:1004E0004FF0000BAC46ACE8C009ACE8C009ACE882
:1004F000C009ACE8C00921F007018D46704710B56E
:100500000446AFF300802046BDE81040FFF785BEEB
:1005100001491820ABBEFEE726000200704700002C
:1005200080B582B001680A68D20614D50022019213
:100530000A68019249680191019902F037FC4CF276
:10054000D80100EBC000C2F2010101EB8000006A9B
:10055000002818BF804702B080BD0000FEE7000001
:1005600080B54CF26810C2F2010000F0B5F880BD11
:1005700080B54CF26810C2F2010000F0ADF880BD09
:1005800080B540F25000C2F2000000F0A5F880BD36
:1005900080B540F25000C2F2000000F09DF880BD2E
:1005A000002804BF03207047006846F20041C4F2EF
:1005B0000001401A18BF03207047000080B54CF2BC
:1005C0005020C2F2010000F0E3FB80BD80B54CF288
:1005D0009010C2F2010000F0DBFB80BD80B54CF250
:1005E000F010C2F2010000F0D3FB80BDD0F800C0D3
:1005F0006FF00F024AF6AB2352FA8CF2CAF6AA2326
:100600000146A2FB0330000905A31B5C40F2FF304A
:100610002CEA00005F2A88BF0430C1E91603704746
:1006200000061016000610168269816AB2F5005F96
:1006300006D06AB9022912D0012914D0D1B90EE02E
:10064000032917D8DFE801F0020B020F01207047E1
:1006500003293CBF012070471CBF00207047C06ABF
:10066000C0F300607047C06AA0F1C070B0FA80F0BB
:1006700040097047002070477047000080B5012096
:1006800000F0CAFC80BD000080B5082000F0C4FC6A
:1006900080BD000080B5102000F0BEFC80BD0000D1
:1006A00080B5202000F0B8FC80BD000072B600BF0D
:1006B000FEE7000080B5FFF773FF032808BF80BD89
:1006C0004CF27001C2F20101342210FB0210006BE7
:1006D000002818BF804780BD2DE9F04F81B0044647
:1006E00000684669D0F804908768D0F80CB0D0F85C
:1006F00010A0D0F81880F10703D1002530071CD4D2
:1007000023E0F90710D00121BA07816009D47807E6
:1007100000F1AA80380700F1B080204600F068FAA6
:1007200002E0204600F076FA0025F80500F184800A
:10073000F80300F1AA80300707D51BF0100004D0A1
:10074000206845F400751021C160700708D51BF0C2
:10075000080005D020680821C160204600F0EEF9AD
:10076000B00706D52068C068800702D0204600F098
:10077000F7F9700607D51AF0100004D0206845F488
:10078000806510210161B00608D51AF0080005D077
:10079000206808210161204600F0F4F9F00606D532
:1007A00020680069800702D0204600F0FDF9B00300
:1007B00008D519F0100005D02068102141602046AE
:1007C00000F004FAF00308D519F0080005D02068FD
:1007D00008214160204600F077FA300440F18F8014
:1007E0005FEA497040F1888006F4807008EA1020C2
:1007F00028435FEA8871014648BF41F00201B20513
:1008000058BF01465FEA48700D4648BF45F00405F1
:10081000700558BF0D4630056ED518F070006BD0CE
:1008200010380009052862D8DFE800F00353565954
:100830005C5F45F008055AE020684FF48071BA0506
:1008400081600AD4780512D4380519D4204600F006
:10085000F3F9F8037FF56FAF17E0204600F0FEF9DB
:10086000F8037FF568AF10E04FF400655DE705F52C
:100870000055F8037FF55FAF07E04FF4805554E76C
:1008800005F58045F8037FF556AF20684FF48031B9
:10089000BA0381600AD478030FD4380313D42046F6
:1008A00000F0EEF930073FF548AF4EE7204600F084
:1008B000F9F930073FF541AF47E705F50045300747
:1008C0003FF53BAF41E705F5803530073FF535AFE4
:1008D0003BE745F010050AE045F0200507E045F04C
:1008E000400504E045F0800501E045F4807520688E
:1008F000816921F0700181612068042141602DB17E
:10090000606A284360622046FFF7D4FE01B0BDE86C
:10091000F08F0000B0B5C8B1044690F8200010B9BF
:10092000204600F071F82068016841F00101016083
:1009300000F054FC054600BF20684168C90707D194
:1009400000F04CFC401B0B28F6D312E00120B0BD98
:10095000016821F00201016000F040FC054600BF83
:100960002068416889070DD500F038FC401B0B2832
:10097000F6D3606A052140F400306062012084F8FB
:100980002010B0BD217E0268012922F0800208BF3C
:1009900080320260617E0268012922F0400208BFB5
:1009A00040320260A17E0268012922F0200208BFC5
:1009B00020320260E17E0268012922F0100218BF95
:1009C00010320260217F0268012922F0080208BF6C
:1009D00008320260617F0268012922F0040208BF28
:1009E00004320260D4E901C2D4E9033561691A43D3
:1009F0002A431143ACF101021143C16100200121DE
:100A0000606284F82010B0BDB0B586B0006846F6CC
:100A10000002C4F2000200219042CDE90411CDE9A8
:100A20000211019136D046F20041C4F20001884221
:100A300040F0828040F24401C2F200010A6843F6AD
:100A40004000C4F20200531C0B6052B90021009117
:100A5000016841F000710160016801F000710091CE
:100A600000990021009150F8101C152441F0080154
:100A700040F8101C50F8100C142500F008000090ED
:100A800000980320019040F20040C4F2020000F5FB
:100A9000006036E043F64000C4F2020000910168B5
:100AA00041F080610160016801F08061009100996E
:100AB00040F24401C2F200010A68531C0B6052B9B3
:100AC00000210091016841F000710160016801F0AE
:100AD0000071009100990021009150F8101C4124F0
:100AE00041F0020140F8101C50F8100C402500F0B5
:100AF0000200009000986020019040F20040C4F293
:100B00000200022102910021039103210491092195
:100B1000059101A900F08EFA28460521002200F077
:100B2000E3FC284600F0DCFC20460521002200F012
:100B3000DBFC204600F0D4FC06B0B0BD80B5FFF76A
:100B40002FFD032808BF80BD4CF27001C2F20101E5
:100B5000342210FB0210C069002818BF804780BDF6
:100B600080B5FFF71DFD032808BF80BD4CF2700162
:100B7000C2F20101342210FB02108069002818BF64
:100B8000804780BD80B5FFF70BFD032808BF80BDFF
:100B90004CF27001C2F20101342210FB0210406AD3
:100BA000002818BF804780BD80B5FFF7F9FC0328F7
:100BB00008BF80BD4CF27001C2F20101342210FB6B
:100BC0000210006A002818BF804780BD80B5FFF77B
:100BD000E7FC032808BF80BD4CF27001C2F201019E
:100BE000342210FB0210806A002818BF804780BDA5
:100BF00080B5FFF7D5FC032808BF80BD4CF270011B
:100C0000C2F20101342210FB0210C068002818BF94
:100C1000804780BD80B5FFF7C3FC032808BF80BDB7
:100C2000342148434CF27001C2F2010108580028F7
:100C300018BF804780BD000080B5FFF7B1FC0328D6
:100C400008BF80BD4CF27001C2F20101342210FBDA
:100C500002100069002818BF804780BD80B5FFF7EB
:100C60009FFC032808BF80BD4CF27001C2F2010155
:100C7000342210FB02104068002818BF804780BD56
:100C800080B5FFF78DFC032808BF80BD4CF27001D2
:100C9000C2F20101342210FB02104069002818BF83
:100CA000804780BD80B5FFF77BFC032808BF80BD6F
:100CB0004CF27001C2F20101342210FB0210806874
:100CC000002818BF804780BD80B5FFF769FC032866
:100CD00008BF80BD4CF27001C2F20101342210FB4A
:100CE0000210C06A002818BF804780BD70B5866DAD
:100CF000044600F073FA94F83510022925D1054610
:100D00002068216C026822F016020260426922F01B
:100D10008002426109B9A16C19B1016821F0080192
:100D20000160016821F00101016000BF20680068D6
:100D3000C0070ED000F052FA401B0628F6D3202040
:100D40006065032084F835000CE080206065012098
:100D500008E0E06D3F2101FA00F0B060012084F866
:100D600035000020002184F8341070BD90F8351053
:100D7000022909D1052180F835100068016821F0A9
:100D8000010101600020704780214165012070470A
:100D9000F0B581B00446002000904CF20000C2F291
:100DA00001000268D4E9166048F2B51337680821DB
:100DB000C1F64E3381403942A2FB03250CD0226894
:100DC00013685B0708D5136823F004031360B16050
:100DD000616D41F00101616501218140394208D016
:100DE00022685269120604D5B160616D41F00201BA
:100DF000616504218140394208D022681268920757
:100E000004D5B160616D41F004016165102181403C
:100E1000394215D020680268120711D5B160026806
:100E20000168520306D4C90506D4016821F00801FF
:100E3000016001E0080342D4216C09B120468847D3
:100E4000E16D202000FA01F23A4244D020680368A4
:100E5000DB0640D5B26094F835300268052B1ED110
:100E600022F016020260426922F080024261226C86
:100E70000AB9A26C1AB1026822F0080202603F208F
:100E80008840B060012084F83500216D00200029E1
:100E900084F8340040D02046884701B0F0BD016896
:100EA000520310D4C90512D4016821F01001016069
:100EB000012084F83500002084F8340007E0A16C9C
:100EC0000029BBD1BCE7080301D4616C00E0E16BF1
:100ED00009B120468847606DF0B1606DC00717D03A
:100EE000052084F835002068A90A026822F0010272
:100EF000026000BF009A01328A42009202D8026862
:100F0000D207F7D1012084F83500002084F834009E
:100F1000E16C09B12046884701B0F0BD2DE9F041F0
:100F2000044600F05BF9C4B10546022084F83500A0
:100F30000020216884F83400086820F0010008606F
:100F400026683068C0070BD000F048F9401B052820
:100F5000F6D903212022032042E00120BDE8F081E0
:100F6000306848F23F01CFF21001251D00EA010C64
:100F70002ECDD4E9050E41EA0C0111431943294352
:100F8000D4E90778084340EA0E01606A394304282F
:100F900041EA080103D1D4E90B231143194331601D
:100FA0007169042821F0070141EA00050CD1D4E958
:100FB0000A1045EA010538B12046FFF735FB18B1A4
:100FC0000121402201200BE020467561FFF70EFB56
:100FD000E16D3F2202FA01F181600022012100202F
:100FE000626584F83510BDE8F081000070B540F20C
:100FF000040604460025C2F2000603E00135102D68
:1010000008BF70BD24FA05F0C007F7D056F82500D8
:10101000002818BF8047F1E780B543F61441C4F2B9
:1010200001010A68024208BF80BD0860FFF7DEFFC9
:1010300080BD00002DE9F04F83B000F13E4202F187
:10104000FF724FEAB22241F600470192C4F2020752
:1010500008224FF0010E00254FF0000A4FF0000863
:10106000B84208BF072200920AE000BF08F1010859
:101070000AF1040AB8F1100F05F1020500F0A4808E
:101080000C680EFA08FB14EA0B09EFD04C6804F068
:10109000030CACF1010EBEF1010F11D803228768D9
:1010A00002FA05F6CA68B743AA403A43826042682A
:1010B000C4F3001722EA0B0207FA08F73A4342602A
:1010C000BCF1030F1CD0C26803238E6803FA05F736
:1010D000BA4306FA05F73A43BCF1020FC2600FD1DA
:1010E0006FF0030202EA580202440AF01C060F23C2
:1010F000176A03FA06F40B69A743B3403B43136234
:10110000026803234F68AB409A4307F00303AB40E8
:101110001A4317F4403F4FF0010E0260A6D00022A0
:1011200043F644030292C4F202031A6843F60044F1
:1011300042F480421A601A68C4F2010402F4804248
:101140000292029A28F003024FF6084B2244CFF68F
:10115000FF7B52F80B300AF00C070F26BE4023EA43
:10116000060C019B009E072B38BF1E4606FA07F7A8
:1011700047EA0C0342F80B30A2684B6842EA0907C1
:1011800043F60C4CDE0258BF22EA0907A760C4F2FE
:10119000010CDCF800209E0242EA090758BF22EA4F
:1011A0000907CCF8007062689E0342EA090758BF3D
:1011B00022EA090767602268DB0342EA090358BF95
:1011C00022EA0903236051E703B0BDE8F08F000075
:1011D000002A08BF090481617047000049F65030B9
:1011E000C2F2010000687047F0B581B0B0B30446A8
:1011F00090F83D0028B9002084F83C00204600F01B
:10120000BFF8242084F83D002068016821F0010126
:101210000160016841F400410160016821F400416E
:10122000016000F02BFA48F28041C0F21E0140F646
:101230000012656888424FF00001C0F23D0248F29A
:10124000A16C4FF0000338BF01219042C0F2010CA5
:1012500038BF0123654538BF0B4613B1012001B0EB
:10126000F0BD4DF68361C4F21B31A0FB0112216871
:101270004FEA924E4B684FF4967623F03F0343EAD1
:1012800092434B6044F6D3530F6A0EFB06F6C1F24D
:101290006203A6FB033627F03F03B709654538BF55
:1012A000970C7A1C1A430A62CA6948F2A0674CF686
:1012B000FF73C0F20107BD4222EA030C0AD80138CD
:1012C0006A00B0FBF2F001306FF31F30042898BFC2
:1012D00004202BE0A368A0F1010E9BB11920684304
:1012E000BEFBF0F00422013062F31F30000512D083
:1012F0009BB119206843BEFBF0F00422013062F379
:101300001F3011E005EB4500BEFBF0F001306FF33C
:101310001F300005ECD1012008E005EB4500BEFBC5
:10132000F0F001306FF31F3040F4004040EA0C0051
:10133000C8610868D4E9072320F0C00010431843AF
:101340000860886848F2FF3204F10C0790438CCFA4
:1013500018431043A6698860C86820F0FF0038432E
:101360003043C860086840F0010008600020202178
:10137000206484F83D10206384F83E0001B0F0BD85
:10138000B0B586B045F200410068C4F20001002407
:1013900088420594CDE903440294019401D006B03B
:1013A000B0BD43F630050094C4F20205286840F051
:1013B00002002860286800F00200009000984FF4B6
:1013C000407001901220CDE9020403200490042013
:1013D000059001F5D83001A9FFF72CFE009428698B
:1013E00040F400102861286900F400100090009873
:1013F00006B0B0BD40F2000049F65031C2F2000024
:10140000C2F2010100780A681044086070470000C9
:1014100080B543F60040C4F20200016841F4007157
:101420000160016841F480610160016841F48071EC
:101430000160032000F068F80F2000F005F800F0CC
:101440002BF8002080BD0000B0B540F20002C2F2CF
:1014500000024CF200011278C2F201014FF47A73DB
:101460000968B3FBF2F20446B1FBF2F1084600F062
:10147000F1FB0F2C4FF001050CD858B94FF0FF309D
:1014800021460022002500F02FF84CF20400C2F2A1
:10149000010004602846B0BD80B582B0002043F64C
:1014A00040010190C4F202014A6842F480424A605D
:1014B0004A6802F480420192019A00900868002272
:1014C00040F08050086008680F2100F080500090C4
:1014D00000986FF0010000F007F802B080BD000036
:1014E00080B501F0A3FD80BD70B514460D460646DB
:1014F00001F0ACFD2946224601F0DAF901463046FA
:1015000001F0ACFD70BD000080B501F0C1FD80BDF3
:101510002DE9F041002800F08B8043F60808C4F262
:1015200002080446D8F8F8030D4600F00700884288
:1015300007D288F8F853D8F8F80300F00700A8425B
:1015400076D12068810717D5410705D5D8F8001056
:1015500041F4E051C8F80010010705D5D8F8001093
:1015600041F46041C8F80010D8F80010A26821F0DA
:10157000F0011143C8F80010C0073FD1D8F8F803B4
:1015800000F00700A84207D988F8F853D8F8F80304
:1015900000F00700A8424BD12068410707D5D8F8D2
:1015A0000010E26821F4E0511143C8F80010000770
:1015B00008D5D8F80000216920F4604040EAC10055
:1015C000C8F8000000F07EF8D8F8001044F6AE62CB
:1015D000C1F30311C0F60002515C4CF2000220FA84
:1015E00001F14CF20400C2F201000068C2F20102F3
:1015F0001160FFF729FF0020BDE8F0816068811EBF
:10160000022907D258F8081C89015CBF0120BDE8F7
:10161000F08110E0012807D158F8081C89035CBF4D
:101620000120BDE8F08106E058F8081C890702D4C3
:101630000120BDE8F081D8F8001021F00301084333
:10164000C8F80000FFF7CAFD064641F2883700BF20
:10165000D8F80000616800F00C00B0EB810F8DD06D
:10166000FFF7BCFD801BB842F2D90320BDE8F08132
:101670004CF20000C2F201000068704780B5FFF72D
:10168000F7FF43F60801C4F20201096844F6BE629E
:10169000C1F38221C0F60002515CC84080BD000049
:1016A00080B5FFF7E5FF43F60801C4F202010968BF
:1016B00044F6BE62C1F34231C0F60002515CC8403C
:1016C00080BD000010B543F60404C4F20204606853
:1016D00000F00C0008280AD0042819BF42F200408C
:1016E000C0F2F40041F60030C0F2B70010BD20682F
:1016F00021682368490241F60031C0F2B70100F0C9
:101700003F02C3F388105CBF42F20041C0F2F40113
:10171000A1FB00010023FEF7A7FD21680222C1F30F
:10172000014102EB4101B0FBF1F010BD2DE9F041A8
:1017300082B0002800F0A2800446007843F600063C
:10174000C007C4F2020643D0B06800F00C000428C1
:1017500005D1306880033BD56068C8BB8EE0B068B7
:1017600000F00C00082802D170684002F1D46568CE
:10177000B5F5A02F0AD0B5F5803F0BD0306820F426
:1017800080303060306820F4802006E0306840F41B
:1017900080203060306840F480303060FFF71EFDFC
:1017A000002D054611D000BF3068800310D4FFF72C
:1017B00015FD401B6428F7D922E100BFFFF70EFD9D
:1017C000401B64284FF0030055D830688003F5D4DF
:1017D000207880071AD5B06810F00C0F09D0B068D7
:1017E00000F00C00082840F08A807068400200F188
:1017F00086803068800702D5E06801283ED13068D5
:10180000216920F0F80040EAC1003060207800072C
:1018100038D4207840074CD4A5695DB3B06800F097
:101820000C00082840F09E80012D27D07068E169E7
:1018300000F480028A4221D1216A00F03F028A42EC
:101840001CD147F6C071626A0140B1EB821F15D10D
:10185000A26A0023CFF6FF7303EBC23200F44031DB
:101860006FF30F02914209D1E16A00F07060B0EBB2
:10187000016F03D1002002B0BDE8F081012002B069
:10188000BDE8F0816069002840F20000C4F2472002
:1018900057D00121C0F8801EFFF7A0FC054600BF0D
:1018A000706F8007B5D4FFF799FC401B0228F7D969
:1018B000A6E0306C10F080580AD100200190306C06
:1018C00040F080503064306C00F0805001900198FE
:1018D00047F20007C4F200073868C00524D438680E
:1018E00040F480703860FFF779FC05463868C00521
:1018F0001AD4FFF773FC401B0228F7D980E0E06898
:10190000002851D00020C4F2472001210160FFF7D8
:1019100065FC0546306880073FF571AFFFF75EFC58
:10192000401B0228F6D96BE0A568052D50D0012D8B
:1019300052D0306F20F001003067306F20F004008B
:101940004DE00021C0F8801EFFF748FC054600BFAF
:10195000706F80077FF55DAFFFF740FC401B0228EA
:10196000F6D94DE00027C4F2472700203866FFF77C
:1019700035FC022D05460BD13068800158D5FFF7A4
:101980002DFC401B02284FF00300F5D973E700BF80
:10199000306880017FF56EAFFFF720FC401B022806
:1019A0004FF00300F4D966E70020C4F2472000217D
:1019B0000160FFF713FC0546306880077FF526AF0E
:1019C000FFF70CFC401B02284FF00300F4D952E74C
:1019D000306F40F004003067306F40F00100306736
:1019E000FFF7FCFB002D054641F2883714D000BFFD
:1019F000306F800713D4FFF7F1FB401BB842F7D9D3
:101A0000032002B0BDE8F081FFF7E8FB401BB842BD
:101A10004FF003003FF62FAF306F8007F4D4B8F1DA
:101A2000000F7FF4F9AE306C20F080503064F3E6A4
:101A300004F11C052FCD08430021CFF6FF7140EAC9
:101A4000821001EBC3316FF30F0140EA05600843D8
:101A5000706001203866FFF7C1FB044630688001E2
:101A60003FF508AFFFF7BAFB001B02284FF0030059
:101A7000F4D900E770B538B10446406A30B10020AF
:101A8000206104F1140007E0012070BD6068B0F52A
:101A9000827F03D004F11C00002101600026A662B1
:101AA00094F8510020B9204684F8506000F03CF8CA
:101AB000022084F8510094E80F0001F48271056857
:101AC00002F4044225F040050560114403F400626D
:101AD0002369114403F002026369114403F0010217
:101AE000A369E569114403F40072114405F038025A
:101AF000256A114405F08002A56A114305F40052DD
:101B000011430160626A042101EA134102F01002EC
:101B100011444160C16921F40061C1610120666521
:101B200084F85100304670BD2DE9F04F87B004466F
:101B300043F200070068C4F201070026B842069687
:101B4000CDE904660396029602D007B0BDE8F08F97
:101B500043F630000196C4F20200416902AD41F43F
:101B600080514161416946F2404801F48051019140
:101B70000199019601684FF0020941F002010160EC
:101B800001684FF0030A01F00201019101990196E9
:101B900001684FF0050B41F0010101600068294622
:101BA00000F00100019001981820029007F55440C0
:101BB000C4F20208CDE90396CDF814A0CDF818B010
:101BC000FFF738FA8020CDE9020904A880E8400C2C
:101BD00007F550402946FFF72DFA4CF29015C2F256
:101BE00001054FF0C06A4FF480694FF40037284672
:101BF000C5E9008AC5E90266C5E90496C5E9066635
:101C0000C5E90876FFF78AF9002818BFFEF74EFDF0
:101C1000E564AC634CF2F01508F11800C2F201055E
:101C20004021C5E9000A05F10800002280E806020B
:101C30002846C5E90522C5E907276A62FFF76EF95C
:101C4000002818BFFEF732FDA564AC6307B0BDE8FD
:101C5000F08F000080B500F095FE80BD002804BF25
:101C60000120704710B5044690F83D0028B90020C7
:101C700084F83C00204600F01FF8022084F83D0064
:101C80002068211D00F0FCFE012084F8460084F845
:101C90003E0084F83F0084F8400084F8410084F856
:101CA000420084F8430084F8440084F8450084F836
:101CB0003D00002010BD000081B0006844F20041EA
:101CC000C4F20101884201D001B0704700200090A9
:101CD00043F64400C4F20200016841F4003101609F
:101CE000006800F400300090009801B070470000D8
:101CF00080B586B044F200410068C4F201010022C0
:101D000088420592CDE903220292019201D006B0E9
:101D100080BD43F630000092C4F20200036843F035
:101D200020030360006800F020000090009840202D
:101D300001900220CDE902020320059001F55040F8
:101D400001A90492FFF776F906B080BDB0B504464C
:101D500090F83C00012804BF0220B0BD0D464FEAB8
:101D6000B2010120032984F83C0037D8DFE801F0F4
:101D7000020A12222068294600F018FF206850F855
:101D8000181F0EE02068294600F042FF206850F836
:101D9000181F16E02068294600F070FF206850F8F0
:101DA0001C1F41F008010160016821F0040101607D
:101DB00029690FE02068294600F094FF206850F858
:101DC0001C1F41F400610160016821F48061016021
:101DD000296909020268114301600020002184F88A
:101DE0003C10B0BD002804BF0120704710B5044668
:101DF00090F83D0028B9002084F83C00204600F00F
:101E00001FF8022084F83D002068211D00F038FEF4
:101E1000012084F8460084F83E0084F83F0084F8EE
:101E2000400084F8410084F8420084F8430084F8BC
:101E3000440084F8450084F83D00002010BD0000F7
:101E4000704700007047000080B500F0AFFF052824
:101E500008BF80BD4CF2D80100EBC000C2F2010106
:101E600001EB80000069002818BF804780BD00009A
:101E7000B0B582B0036804461868D9685A6900F0A2
:101E80002F05202D01F0200505D125B1204600F0B9
:101E9000B7FF02B0B0BD5FEA007C1EBF02F0010ECA
:101EA00001F4907212EB0E024AD1226B0840C10677
:101EB0003DD5012A3BD10020019018680190586857
:101EC000019001985869400642D4A08DE18DE28DC1
:101ED000002A1CBF401A5FEA004101D102B0B0BD28
:101EE000216851E8031F226821F4907142E803132E
:101EF000002BF5D1216851E8051F226821F001016E
:101F000042E80513002BF5D1202184F8421000216E
:101F1000216300BF216851E8031F226821F01001EE
:101F200042E80313002BF5D10221616354E001065E
:101F300054D44006D2D5204600F02CFF02B0B0BDEC
:101F4000C20718BF11F480725DD1420761D467E007
:101F5000E06B016849688AB2002A44D0A38D9A4296
:101F600041D2E185C069B0F5807F30D0206850E86B
:101F7000030F216820F4807041E80302002AF5D1A4
:101F8000206850E8050F216820F0010041E80502B3
:101F9000002AF5D1206850E8050F216820F04000A4
:101FA00041E80502002AF5D1202084F842000020F3
:101FB000206300BF206850E8030F216820F0100064
:101FC00041E80302002AF5D1E06BFEF78FFE022004
:101FD0006063A08DE18D401A81B20FE0204600F0D1
:101FE000E1FF02B0B0BDA18D91427FF477AFC0692F
:101FF000B0F5807F7FF472AF022060632046FFF768
:1020000021FF02B0B0BD626C42F00102626442077F
:1020100006D5BEF1000F03D0626C42F0020262648A
:10202000820706D5BEF1000F03D0626C42F00402B5
:102030006264BCF1000F06D55EEA050203D0626C53
:1020400042F008026264626C002A3FF447AF084025
:10205000800602D5204600F0D3FE20684069616CFE
:1020600000F0400001F00801401827D0204600F0A1
:1020700069FE2068406940061BD500BF206850E813
:10208000050F216820F0400041E80502002AF5D143
:10209000E06B70B142F63551C0F600010165FEF704
:1020A00065FE00283FF41AAFE06B016D884702B06F
:1020B000B0BD2046FFF7C8FE02B0B0BD2046FFF716
:1020C000C3FE0020606402B0B0BD0000002804BF61
:1020D0000120704710B5044690F8410028B900204F
:1020E00084F84000204600F021F8242084F84100C4
:1020F0002068C16821F40051C160204600F0E4FE70
:102100002068016921F490410161416921F02A01AF
:102110004161C16841F40051C16000202021606428
:1021200084F8411084F84210606310BD2DE9F0433B
:1021300087B00446006840F6FF71C4F2010188428E
:102140004FF000010691CDE90411CDE902115FDCE9
:1021500044F20041C4F20001884200F0B58044F628
:102160000001C4F20001884240F00681002643F6D7
:1021700030000196C4F20200016941F4802101613E
:10218000016901F48021019101990196016841F0F2
:1021900004010160006802A900F0040001900198A8
:1021A0004FF4406002900220CDE903060320059021
:1021B000072006900020C4F2020000F50060FEF740
:1021C00039FF4CF2502546F22800C2F20105C4F254
:1021D00002004FF000614FF480624FF4807385E895
:1021E00043002846C5E90362C5E90566C5E9073627
:1021F0006E62FEF793FE002818BFFEF757FA2720FD
:1022000005210022E563AC63FFF76EF9272056E055
:1022100041F20041C4F20101884200F0828041F2A3
:102220000001C4F20101884240F0A680002643F676
:1022300030000196C4F202004169002441F010010F
:1022400041614169C4F2020401F010010191019958
:102250000196016802AD41F00201016001684FF092
:10226000020801F0020101910199019601684FF005
:10227000030941F0010101600068072700F0010037
:10228000019001988020029004F580602946CDE9F4
:102290000386CDF814900697FEF7CCFE4FF400703D
:1022A000CDE9020820462946CDE904690697FEF7E4
:1022B000C1FE252005210022FFF716F92520FFF792
:1022C0000FF907B0BDE8F083002043F6300101901C
:1022D000C4F202010A6942F400320A610A6902F496
:1022E00000320192019A01900A6842F008020A60E5
:1022F000096801F008010191019960210291022110
:10230000CDE9031003200590072006900020C4F2B9
:10231000020000F5406002A9FEF78CFE07B0BDE8A0
:10232000F083002043F630010190C4F202014A69B3
:1023300042F020024A614A6902F020020192019AA9
:1023400001900A6842F040020A60096801F0400109
:10235000019101994FF4844102910221CDE90310CA
:1023600003200590082006900020C4F2020000F52A
:10237000C05002A9FEF75EFE07B0BDE8F083000082
:1023800080B500F013FD052808BF80BD4CF2D801D0
:1023900000EBC000C2F2010101EB8000C068002820
:1023A00018BF804780BD000080B500F0FFFC052805
:1023B00008BF80BD4CF2D80100EBC000C2F20101A1
:1023C00001EB80004068002818BF804780BD0000F6
:1023D000FEE7000010B54CF2681046F20041C2F270
:1023E0000100C4F200010322002380E80E0000F186
:1023F0000C014FF4102C4FF4001E4FF0807481E854
:1024000008504FF4807184618183FEF783FA0028BD
:1024100018BFFEF74BF910BD10B540F2500046F65C
:102420000001C2F20000C4F200010322002380E890
:102430000E0000F10C014FF4102C4FF4001E4FF071
:10244000807481E808504FF4807184618183FEF7C5
:1024500061FA002818BFFEF729F910BD80B582B0D7
:10246000002043F630010190C4F202010A6842F4F0
:1024700080020A600A6802F480020192019A0090C8
:102480000868002240F4001008600868052100F484
:102490000010009000980C20FFF726F80C20FFF7A2
:1024A0001FF83A2005210022FFF71EF83A20FFF717
:1024B00017F83B2005210022FFF716F83B20FFF715
:1024C0000FF802B080BD000080B542F67D1044F6E2
:1024D000C862C0F60000C0F60002002100F048FE0D
:1024E00040F24C01C2F20001086080BD2DE9F04FBE
:1024F00087B0002443F630000694CDE90444CDE9CA
:1025000002440194C4F20200016840F2000941F063
:10251000020101600168C4F2020901F002010191A7
:1025200001990194016809F5C05A41F04001016028
:102530000168002201F040010191019901940168B4
:10254000402741F001010160016801F001010191A2
:1025500001990194016841F008010160016801F0EE
:102560000801019101990194016841F004010160A1
:10257000016801F00401019101990194016841F0A1
:1025800080010160016801F08001019101990194CD
:10259000016841F0200101600068402100F0200046
:1025A000019001985046FEF713FE09F5E0552846C4
:1025B0004FF4A0510022FEF70BFE28464FF40061B5
:1025C00001220126FEF704FE4846102101224FF0A9
:1025D000100BFEF7FDFD09F5806840460121012240
:1025E000FEF7F6FDCDE9027602AF50463946CDE959
:1025F0000464FEF71FFD4FF4E050CDE902062846C3
:102600003946CDE90464FEF715FD082002904FF429
:10261000041450463946CDE90346FEF70BFD484603
:102620003946CDE902640496FEF704FD4846394672
:10263000CDE902B6CDE90466FEF7FCFC302002A924
:1026400051C109F500603946FEF7F4FC40463946B1
:10265000CDE90266CDE90466FEF7ECFC0620052113
:102660000022FEF741FF0620FEF73AFF0920052170
:102670000022FEF739FF0920FEF732FF0A2005216C
:102680000022FEF731FF0A20FEF72AFF172005215E
:102690000022FEF729FF1720FEF722FF07B0BDE852
:1026A000F08F000080B540F2780045F20041C2F2A0
:1026B0000000C4F2000148F2A06200234FF4804CF5
:1026C000C0F2010280E80E00C0E9033CC0E9053316
:1026D000C0E90733FEF788FD002818BFFDF7E6FFC5
:1026E00080BD0000B0B54CF2B02043F20001C2F250
:1026F0000100C4F201014FF48272002380E80E0051
:1027000000F10C014FF0020C4FF0010E4FF4007479
:10271000182581E808500A21C0E90645C0E90833B8
:10272000C0E90A31FFF7A6F9002818BFFDF7BEFF80
:10273000B0BD000080B588B040F2CC0044F2004249
:102740000021C2F20000C4F2010241F28833079175
:10275000CDE90511CDE90311CDE90111C0E9002151
:10276000C0E9021301618161FFF778FA002818BF00
:10277000FDF79CFF40F2CC00C2F20000FFF732FBF5
:10278000002818BFFDF792FF602001900020CDE9DE
:102790000200059040F2CC00C2F2000001A9002224
:1027A000FFF7D4FA002818BFFDF780FF40F2CC00F5
:1027B000C2F20000FFF79CFA08B080BD80B54CF271
:1027C000083041F20001C2F20100C4F2010100230D
:1027D0004FF00C0C4FF4E13280E80E00C0E90333F7
:1027E000C0E905C3C361FFF771FC002818BFFDF7FE
:1027F0005DFF80BD80B540F2141044F20041C2F28A
:102800000000C4F2000100234FF00C0C4FF4E13241
:1028100080E80E00C0E90333C0E905C3C361FFF7D8
:1028200055FC002818BFFDF741FF80BD10B54CF2E4
:10283000503044F6000C48F2A062C2F20100C4F22B
:10284000000CC0F201024FF4805300214FF4806E5F
:102850000C24C0E900C2C0E90231C0E904E4C0E9C7
:102860000611FFF733FC002818BFFDF71FFF10BD4E
:1028700080B540F25C1041F20041C2F20000C4F2A7
:10288000010100234FF00C0C4FF4E13280E80E0000
:10289000C0E90333C0E905C3C361FFF717FC002893
:1028A00018BFFDF703FF80BDFEE70000FEE7000054
:1028B00000F0070080F00703042B28BF04234FF02B
:1028C000FF3C03380CFA03F338BF002099438140E2
:1028D0000CFA00F022EA00000843704700000000F4
:1028E000EFF30980BFF36F8F154B1A681EF0100FBE
:1028F00008BF20ED108A20E9F04F10602DE9090093
:102900004FF0500080F31188BFF34F8FBFF36F8FEC
:1029100001F046FC4FF0000080F31188BDE809008B
:1029200019680868B0E8F04F1EF0100F08BFB0EC4F
:10293000108A80F30988BFF36F8F704700BF00BF14
:10294000A4010020000000000000000000000000C2
:10295000074B19680868B0E8F04F80F30988BFF3A7
:102960006F8F4FF0000080F31188704700BF00BFE9
:10297000A401002080B500F083FB80BD012000F0A1
:10298000B9FBFBE7B0B501380024B4EB106F1CBFF6
:102990000120B0BD4EF21005CEF2000568604FF088
:1029A000FF300F2100F05AFB0720AC602860204662
:1029B000B0BD000080B5FEF71DFD02F01DF8012836
:1029C00018BF01F0C5FC80BD70B592B006AC2046C2
:1029D0003021FDF740FD002543F640000595CDE987
:1029E0000355CDE901550095C4F2020001680226A5
:1029F00041F080510160006800F080500090009824
:102A000047F200000095C4F20000016841F48041E3
:102A10000160006800F4804000900098012006905A
:102A20004FF4803007904FF480000D9006200E90F8
:102A3000A820CDE90F060420119020460C96FEF741
:102A400075FE88B90F20CDE901064FF4A05004901F
:102A50004FF48050059001A805210395FEF758FD1D
:102A6000002804BF12B070BDFDF720FE4EF688505E
:102A7000CEF20000016841F470010160704700006F
:102A8000B0B540F6FF3E0568C4F2000E40F2004CBF
:102A90007045C4F2010C0FDCB0F1804F19D040F248
:102AA0000043C4F20003984213D040F60003C4F27E
:102AB000000398420DD011E040F60043C4F2000339
:102AC000984206D0604504D00023C4F20103984226
:102AD00004D14B6825F0700243EA020541F6FF730A
:102AE000C4F2000398420DDC70451FDCB0F1804F4A
:102AF00041D040F20043C4F2000398423BD040F67C
:102B0000000321E043F6FF73C4F20103984220DC86
:102B100042F20003C4F2000398422CD00023C4F216
:102B20000103984227D0604525D029E040F60043B4
:102B3000C4F2000398421ED041F60003C4F2000321
:102B4000984218D041F60043C4F20003984212D0D4
:102B500016E044F20003C4F2010398420BD044F69D
:102B60000003C4F20103984205D044F20043C4F2CA
:102B70000103984204D1CB6825F4407243EA020570
:102B80000A688C684B69C46240F480648262644560
:102B900004BF09690163026825F0800142F0040264
:102BA00019430260012242610160B0BDB0B5026A02
:102BB000036A40F2004523F001030362D0F804E009
:102BC000D0F818C08C6822F0020240F48063C4F28E
:102BD0000105AB4242EA040205D1CC6822F00C02A6
:102BE00024F0040422430C68AB4207D1D1E9055319
:102BF0002EF4407E45EA0E0545EA030E2CF07303E1
:102C00002343C0F804E08361496841630262B0BDB8
:102C100070B5026A036A40F2004423F010030362B5
:102C2000D0F804E0D0F818C08D6822F0200240F4FB
:102C30008063C4F20104A34242EA051207D1CD68C1
:102C40006FF0400622F0C00206EA05152A430D681F
:102C5000A34207D1D1E905642EF4406343EA860319
:102C600043EA840E2CF4E64343EA0523C0F804E06B
:102C7000836149688163026270BD000070B5026AB9
:102C8000036A40F2004423F480730362D0F804E046
:102C9000D0F81CC08D6822F4007240F48063C4F246
:102CA0000104A34242EA052207D1CD6840F2FF4663
:102CB0002D0222F44062B5432A430D68A34207D196
:102CC000D1E905642EF4405343EA061343EA041E97
:102CD0002CF073032B43C0F804E0C3614968C1635F
:102CE000026270BD70B5D0F820C0026A40F20046A2
:102CF00022F4805202624268C3690C68D1F808E08D
:102D000040F48065C4F20106B54204D14D6922F455
:102D1000804242EA851223F4E64343EA04234260F8
:102D2000C3612CF40056496846EA0E32016402621F
:102D300070BD000080B5806B0021C185FFF784F86D
:102D400080BD0000016851E8031F026821F4907102
:102D500042E80313002BF5D1016851E8051F026812
:102D600021F0010142E80513002BF5D1016B012987
:102D70000AD100BF016851E8031F026821F0100169
:102D800042E80313002BF5D1202180F842100021E6
:102D90000163704780B50168CA6822F04002CA60CA
:102DA000202180F84110FFF7FFFA80BD006840F64F
:102DB000FF71C4F20101884210DC44F20041C4F208
:102DC0000001884204BF0120704744F60001C4F2AC
:102DD0000001884204BF022070470FE041F2000169
:102DE000C4F20101884204BF0020704741F2004153
:102DF000C4F20101884204BF0320704705207047D8
:102E000080B582B090F8421022291ED18268B2F5B6
:102E1000805F02D1016900294AD0816AB2F5805FE2
:102E200007D00AB9026922B10268526802F07F0233
:102E300001E0026852680A700121826A11448162CD
:102E4000C18D01390A04C18501D002B080BD01687D
:102E5000CA6822F02002CA60CA6822F48072CA607E
:102E60004A6922F001024A61202180F842100021C3
:102E70004163026B012A23D1016300BF016851E85D
:102E8000031F026821F0100142E80313002BF5D163
:102E900001680A68D20606D5002201920A680192EA
:102EA000496801910199818DFEF7CCFF02B080BD88
:102EB0000168826A49686FF35F2111800221BCE7D3
:102EC000FFF75EFA02B080BD10B504460068D4E991
:102ED00002C22369016921F4405111430161626911
:102EE00043EA0C01E3691143C268194349F20C63D8
:102EF0009A431143C1604169A26921F4407141F2D2
:102F00000043114340F48062C4F201039A424161DC
:102F100002D1FEF7C5FB01E0FEF7B0FBE169636893
:102F20001922B1F5004FA0FB02011CD15A00DB0FA2
:102F3000FDF79AF948F21F51C5F2EB11A0FB0123EE
:102F40005A096FF0630302FB0300322303EBC00056
:102F5000A0FB01014FF4F87000EA111000EB021021
:102F6000C1F342111AE09A009B0FFDF77DF948F278
:102F70001F51C5F2EB11A0FB01235A096FF0630347
:102F800002FB0300322303EB0010A0FB0101F02041
:102F900000EA511000EB0210C1F34311226808430C
:102FA000906010BD90F84110212923D18168B1F5BE
:102FB000805F01D1016931B1016A02684B1C036273
:102FC0000978516007E0016A036831F8022B6FF35A
:102FD0005F225A600162C18C01390A04C18418BFA2
:102FE00070470068C16821F08001C160C16841F08C
:102FF0004001C1607047000010B54CF20834C2F2C5
:1030000001042046FEF734FF2046FDF789FA10BD83
:1030100010B54CF25034C2F201042046FEF728FFEE
:103020002046FDF77DFA10BDFEE70000002848BFEE
:10303000704700F01F01012202FA01F14EF2001266
:103040004009CEF2000242F8201070474EF60C50B4
:10305000CEF200000068C0F3022070474EF6145311
:1030600000F00F02CEF2000309011A4400F16043A0
:10307000B0F1FF3FC8BF03F5644211707047000014
:103080004EF61F50CEF20000002101707047000084
:103090004EF60C51CEF200010A684FF6FF031A40BB
:1030A00060F30A2242F0806040F0FD7008607047D3
:1030B000FEF7AEF9FFF788FCFFF718FAFFF7CEF935
:1030C000FFF788F9FFF7A8F9FFF70CFBFFF732FBD2
:1030D000FFF7ACFBFFF772FBFFF78CFBFFF7C8FBBA
:1030E000FFF7E0FA00F016F8FFF7EEF900F026F827
:1030F000FEE70000EFF3058100291CBF6FF005001B
:103100007047002804BF0020704780B500F074FFAE
:10311000002080BDEFF3058000281CBF6FF0050084
:10312000704740F24800C2F200000168002911BF58
:103130004FF0FF30012101600020704710B5EFF320
:10314000058000281CBF6FF0050010BD40F2480448
:10315000C2F20004206801281CBF4FF0FF3010BDF0
:10316000FFF708FC0220206000F0C0FF002010BD27
:1031700070B584B08E46002100280391EFF30581DD
:1031800046D0002944D1FAB19369002B08BF182317
:10319000382B16D81179C90713D15569946811686D
:1031A0004FEA950C002D08BF4FF0800CFCB1D6689B
:1031B0005C2E1BD3D5B11569C5B10024012555B9C5
:1031C0001BE0002004B070BD0124002118234FF043
:1031D000800C00258DB1946812690294CDE900320B
:1031E0006246734601F0CCFB039011E00CB9D46841
:1031F0009CB100250024002DEDD14CB103AC00930F
:103200001FFA8CF27346019401F086FB012802D16B
:10321000039804B070BD0020E6E71469B4FA84F4A2
:103220006409D6E7F0B581B00D4649F6084140F291
:10323000A416C2F20101C2F200060F68316804460A
:10324000081D00F061FD601C0AD14DB13068011D00
:103250004CF6E470C2F2010000F0B2FD01B0F0BD26
:103260003068E41944600AD340F2A810C2F20000AA
:1032700000683168043100F085FD01B0F0BD4CF20A
:103280009040C2F2010000683168043100F07AFD1C
:103290004CF69070C2F2010001688C4238BF0460A5
:1032A00001B0F0BD70B5044600F0A2FD4CF6F80088
:1032B000C2F20100016840F2A41501310160C2F2BE
:1032C0000005296849F60446C2F2010641B130689A
:1032D00060B92868E16AC06A884298BF2C6005E03E
:1032E0002C600068012801D100F0C4F94CF60010F0
:1032F000C2F2010001680131016061644CF6041101
:10330000C2F20101E06A0A68904288BF08604CF28C
:10331000984100EB8000C2F2010101EB8000211D09
:1033200000F04EFD00F088FD306880B12868E16A49
:10333000C06A884228BF70BD4EF60450CEF200002D
:103340004FF080510160BFF34F8FBFF36F8F70BD9F
:1033500070B582B000F04CFD4DF20C06C2F20106D1
:10336000306850BB4CF66474C2F20104204600F091
:10337000F9FC49F6B435C2F20105284600F0F2FC2A
:103380004CF28C40C2F20100046040F2AC10C2F278
:1033900000004CF298324CF2384305600025C2F22E
:1033A0000102C2F201030A201021009500F0E8FF9B
:1033B000306010B103A100F0E9FD00F03DFD02B066
:1033C00070BD00BF546D725100000000F0B581B0B7
:1033D00049F65435C2F201052868E0B14CF6F8769A
:1033E0004CF6F807C2F20106C2F2010700F000FD38
:1033F000F068C468201D00F087FC38680138386028
:1034000028680138286000F017FD204600F058F8C1
:1034100028680028EAD101B0F0BD000080B5026C38
:10342000002A08BF80BDD0E902C31344C3606345CE
:1034300024BF0368C360C36808461946FCF78CFFC5
:1034400080BD000070B5866B036C0446E3B1154681
:103450001AB3E0681A46FCF77FFFE168206C226827
:10346000091A9142E16003D2A16840420844E06039
:10347000A81EB0FA80F040093146002E18BF012185
:103480000840361A002516E02068002598B9A06883
:1034900001F076FBA56005460DE060681A46FCF772
:1034A0005BFF216CD4E90102002508446060904272
:1034B00024BF20686060711C2846A16370BD0000B5
:1034C00010B5044690F85900022808BF10BD012825
:1034D00003D030B9206B00F0C7FC204600F0C4FCDC
:1034E00010BD4FF0500080F31188BFF36F8FBFF312
:1034F0004F8F00BFFEE700004CF28C41C2F2010189
:1035000009680A68B2FA82F35B090360002A0EBFF9
:103510000020C8680068704740F2B010C2F2000096
:10352000C21D22F0070210F0070CA0EB020318BF27
:1035300010464CF6DC72C2F201020021C2E9000121
:1035400049F69912C0F20102BCF1000F18BF1A44EB
:103550000244083A4CF2944322F00702C2F20103FB
:103560001A60C2E90011111A1A68C0E900214CF66C
:103570008C70C2F20100016049F6E030C2F2010035
:10358000016049F6C830C2F20100012101707047A4
:103590004CF298444EF60455C2F20104CEF20005F6
:1035A0004FF08056FFF712FF20680228FAD32E60F2
:1035B000BFF34F8FBFF36F8FF4E70000B0B5049DEA
:1035C000002914BF2A602D60C5E90F01284601219A
:1035D0001C4600F021FF85F84C40B0BD2DE9F047B6
:1035E0000A9C8246206B16460F46DDE90859910079
:1035F000A5229846FCF727FF206B00EB8600A0F180
:10360000040020F007067FB104F13400002100BF60
:103610007A5C42547A5C1AB10F2901F10101F7D3A7
:10362000002084F8430002E0002084F834000027E2
:10363000201D372D28BF3725E562C4E9135700F058
:103640009DFB04F1180000F099FBC5F13800A06162
:1036500030465146424624616462676584F858707A
:1036600000F03EFBB9F1000F206018BFC9F8004020
:10367000BDE8F087B0B54CF298450024C2F20105D0
:10368000281900F06FFB1434B4F58C6FF8D14CF6A8
:103690007874C2F20104204600F064FB49F6CC3590
:1036A000C2F20105284600F05DFB49F6F030C2F297
:1036B000010000F057FB4CF6F870C2F2010000F078
:1036C00051FB4CF6E470C2F2010000F04BFB4CF2EF
:1036D0009040C2F20100046040F2A810C2F2000063
:1036E0000560B0BD80B54CF6DC72C2F2010200BFCD
:1036F000114612688242FBD3D1F804C001EB0C03DF
:10370000834203D14068604448600846D0F804C052
:1037100000EB0C03934201D013460BE04CF29443B0
:10372000C2F201031B689A4204D0D2E9003E0EEBBC
:103730000C0242608142036018BF086080BD000037
:1037400080B58C46014641F804CF9445006108D904
:103750009A4201D29C4511D24CF28C40C2F2010037
:1037600007E08069D21A824208D240F2AC10C2F25D
:103770000000006800F006FB002080BD012080BD35
:1037800010B5044600F034FBA06BB0FA80F0440999
:1037900000F052FB204610BD10B5044600F028FB97
:1037A000A06BE16B401AB0FA80F0440900F044FBD2
:1037B000204610BD08480068006880F308884FF074
:1037C000000080F3148862B661B6BFF34F8FBFF379
:1037D0006F8F00DF00BF00BF08ED00E070B582B062
:1037E0004CF28C42C2F2010212680546D2680E46C3
:1037F000D468201D00F088FA94F82800410704D40A
:1038000000F0FE0084F8280010E0A069324641195B
:1038100020462B46FFF794FF40B1002620460021AA
:103820002A460023009601F001FB20B1216A2046C0
:10383000884702B070BD4FF0500080F31188BFF38D
:103840006F8FBFF34F8F00BFFEE700002DE9F041FF
:1038500086B04DF20C07C2F20107386802A90022B7
:103860004FF0000800F052FF00286AD001AC02AD12
:103870000BE000F0FE0086F8280000BF38682946FB
:10388000002200F043FF00285BD00298B0F1FF3F18
:1038900003DCDDE903200599904702980028EDD468
:1038A000049E706910B1301D00F02EFA204600F021
:1038B000B3F802990929E1D80246DFE801F00808C7
:1038C00008052A390808052A96F82800D1E796F84D
:1038D0002800039BB16940F0010086F828001944D4
:1038E0003046FFF72DFF0028C8D0316A30468847A0
:1038F00096F828004007C1D50398B16900230A183B
:1039000030460021CDF8008001F090FA0028B5D1B2
:1039100023E096F8280040F00101039886F828106B
:10392000B06188B1811830461346FFF709FFA5E75B
:1039300096F8280081073FF59CAF304600F094FAD6
:103940009CE706B0BDE8F0814FF0500080F311888D
:10395000BFF36F8FBFF34F8FFEE74FF0500080F340
:103960001188BFF36F8FBFF34F8F00BFFEE70000DA
:1039700070B582B00E46044600F00AFC01A800F0C3
:103980004BF8019919B101F08DF902B070BD0546EF
:103990004EB9A54207D301F085F920462946FFF725
:1039A0001DFF02B070BD4EB140F2AC10C2F200007B
:1039B00000680068B0FA80F0420900E000224DF291
:1039C0000C00C2F201000068611B00F0F3FA01F084
:1039D00069F90028D9D14EF60450CEF200004FF01C
:1039E00080510160BFF34F8FBFF36F8F02B070BD86
:1039F0004CF29040C2F201000168096821B10068F0
:103A0000C068C068406801E04FF0FF304CF690712C
:103A1000C2F201010860704770B5044601F000F879
:103A20004CF28846C2F2010631680546884203D24C
:103A300000F008F8012000E00020206028463560F2
:103A400070BD00002DE9F04182B04CF28C47C2F20B
:103A500001073868016891B34FF0000809E000BF22
:103A6000606038682946246100F08CF93868016884
:103A700029B3C068C4680668251D284600F044F9CB
:103A8000216A2046884794F828004007EED5A069AF
:103A90003044B042E4D82046002132460023CDF81D
:103AA000008001F0C3F90028E0D14FF0500080F30E
:103AB0001188BFF36F8FBFF34F8F00BFFEE740F257
:103AC000AC11C2F200010A6808603A6002B0BDE8B9
:103AD000F081000081B0002000904CF20800C2F29A
:103AE000010000684FF0500181F31188BFF36F8F20
:103AF000BFF34F8F013001D0FEE700BF00980028D0
:103B0000FCD001B07047000082B001AC2046FFF746
:103B1000F3FC0199FFF72CFFFFF798FEF6E7000092
:103B2000F0B581B0044600F063F994F94560012EC8
:103B30000FDB04F1240500BF286850B1284601F0CE
:103B400069F8002818BF00F08FFA70B2013E012812
:103B5000F2DCFF2684F8456000F06EF900F048F9C9
:103B600094F94470012F0EDB04F11005286850B160
:103B7000284601F04FF8002818BF00F075FA78B217
:103B8000013F0128F2DC84F8446000F055F901B0EF
:103B9000F0BD00002DE9F04381B0044600F0F8FAD2
:103BA0004CF29446C2F201063068002808BFFFF7C5
:103BB000B3FC49F6C838C2F2010898F800000028A2
:103BC00018BF4FF0004020420DD0002401F06AF8E9
:103BD00060071ED04FF0500080F31188BFF36F8F45
:103BE000BFF34F8FFEE7C4B114F0070004F10801E2
:103BF0001EBF081A00F108015FEA41700ED04FF0B5
:103C0000500080F31188BFF36F8FBFF34F8F00BF59
:103C1000FEE7204601B0BDE8F083002149F6E03917
:103C2000C2F20109D9F800004A1E8242CDD24CF6F8
:103C3000DC70C2F2010005682F4657F8042F8A4253
:103C400011D22B685BB100BF1F4657F8042F2846DE
:103C50001D468A4207D22B68002BF5D103E04CF6B3
:103C6000DC70C2F2010033689D42AED004682B685C
:103C7000521A112A036010D36818430709D04FF075
:103C8000500080F31188BFF36F8FBFF34F8F00BFD9
:103C9000FEE742603960FFF725FD4CF68C7039680D
:103CA000D9F80020C2F201000368511A9942C9F8FC
:103CB000001038BF016098F80000396800284FF004
:103CC000000018BF41F00041286049F6EC30C2F214
:103CD0000100026808343960511C016076E7000079
:103CE000034643F6D520C0F600004FF0807C21F05B
:103CF000010103E903106FF0020043F8240CA3F163
:103D0000440043F8202C7047D0E9013201699A60E1
:103D1000D1F804C082688445536008BF4A6000221D
:103D20000261086801380860086870474CF608337B
:103D3000C2F2010303604CF60810C2F201000860F1
:103D4000802010607047000049F65833C2F201032A
:103D500003604CF66430C2F2010008604FF48070DA
:103D6000106070474FF0FF31024642F8081F0021F3
:103D70004260C0E903220160704700000021016138
:103D80007047000080B5D1F800C01CF1010207D0D7
:103D900000F108039E465B681A686245FAD901E0A3
:103DA000D0F810E0DEF8042008614A609160C1F8A4
:103DB00008E0CEF8041001680131016080BD000008
:103DC000D0F800C0436808619A684B608A609A68BE
:103DD000996051600CF1010101607047DFF80C003F
:103DE000016841F470010160704700BF88ED00E098
:103DF0004FF0500080F31188BFF36F8FBFF34F8FE8
:103E00004CF20800C2F2010001684A1C026001B1D4
:103E100070474EF60450CEF200000068000608BF5E
:103E200070474FF0500080F31188BFF36F8FBFF3DE
:103E30004F8F00BFFEE700004CF20800C2F2010005
:103E4000016839B10139016018BF7047002080F363
:103E5000118870474FF0500080F31188BFF36F8FC7
:103E6000BFF34F8FFEE70000B0B5002808BFB0BD1C
:103E7000044649F6C830C2F20100007854F8041C28
:103E8000002818BF4FF0004008420CD0A4F10805EC
:103E90002A6892B14FF0500080F31188BFF36F8F02
:103EA000BFF34F8FFEE74FF0500080F31188BFF350
:103EB0006F8FBFF34F8F00BFFEE721EA000044F889
:103EC000040C00F065F949F6E031C2F2010154F842
:103ED000040C0A68104408602846FFF703FC4CF6FF
:103EE0009470C2F2010001680131016000F0DAFE55
:103EF000B0BD00004EF21000CEF2000000210160C3
:103F000081604CF20001C2F20101096844F6D3520B
:103F1000C1F26202A1FB02124FF0FF3101EB9211DC
:103F20004160072101607047EFF30580102814D32A
:103F30004EF2F031CEF20001405C49F64931C2F256
:103F400001010978884208D24FF0500080F31188AF
:103F5000BFF36F8FBFF34F8FFEE74EF60C50CEF2DC
:103F6000000049F64C310068C2F20101096800F412
:103F7000E060884298BF70474FF0500080F311888E
:103F8000BFF36F8FBFF34F8FFEE700004CF69C7CB2
:103F90000022C2F2010C00BF5CF8323023B10132C2
:103FA000082A08BF7047F7E70CEBC2034CF8321041
:103FB0005860704770B515460E460446FFF718FF67
:103FC00094F84400FF2804BF002084F8440094F8CB
:103FD0004500FF2804BF002084F84500FFF72CFFB0
:103FE000A06B28B904F1240031462A4600F05EF89F
:103FF0002046FFF795FD70BD10B5D8B104464CF6CC
:10400000FC00C2F20100006848B14FF0500080F39C
:104010001188BFF36F8FBFF34F8F00BFFEE700F033
:10402000B7F820460021FFF7FDF800F03BFE00281E
:1040300018BF10BD4EF60450CEF200004FF0805174
:104040000160BFF34F8FBFF36F8F10BD49F6E831AA
:10405000C2F201010968016049F60841C2F201019A
:10406000096841607047000049F61040C2F2010043
:10407000012101607047000010B568B10C4640F2A4
:10408000A411C2F2000109681831FFF77BFE204637
:104090000121FFF7C7F810BD4FF0500080F31188E1
:1040A000BFF36F8FBFF34F8FFEE70000B0B590B145
:1040B0000D4640F2A411C2F20001096814461831FD
:1040C000FFF77EFE002C18BF4FF0FF352846214633
:1040D000FFF7A8F8B0BD4FF0500080F31188BFF390
:1040E0006F8FBFF34F8F00BFFEE7000010B586B0A3
:1040F000002405A804A903AACDE90444FFF716FE8D
:10410000DDE9032005990023CDE9010143F2915037
:10411000C0F600001CA1009400F032FC49F6E43126
:10412000C2F20101086010B100F046FE0446601CB6
:1041300020D0012C1CD14FF0500080F31188BFF328
:104140006F8FBFF34F8F4CF69070C2F201004FF0AB
:10415000FF31016049F60440C2F201000121016013
:1041600049F60840C2F201000021016000F066F843
:1041700006B010BD4FF0500080F31188BFF36F8F71
:10418000BFF34F8FFEE700BF49444C4500000000DD
:104190004CF6FC00C2F20100016801310160704779
:1041A0004CF6FC00C2F20100006830B149F6104044
:1041B000C2F2010001210160704749F61040C2F2CD
:1041C000010000214CF6041C0160C2F2010CDCF875
:1041D00000104CF2984201EB8103C2F2010252F846
:1041E000230048B902EB8300A0F11403D9B153F8BE
:1041F000140901390028F9D001EB810002EB80029B
:1042000052F8040F4368101D8342136001D15868AF
:104210001060106840F2A412C068C2F20002106080
:10422000CCF8001070474FF0500080F31188BFF3B6
:104230006F8FBFF34F8F00BFFEE7000080B582B0E5
:104240004EF20040CEF200004CF27021C4F20F1189
:10425000D0F800294B1C9A4209D14FF0500080F34E
:104260001188BFF36F8FBFF34F8F00BFFEE7D0F809
:1042700000298A4209D14FF0500080F31188BFF322
:104280006F8FBFF34F8F00BFFEE7017849F64932C9
:104290000191FF2101700178C2F201028DF8031033
:1042A0009DF8031001F05001117049F64C31C2F233
:1042B000010107220A609DF90320B2F1FF3F0CDCE7
:1042C0000A6800BF9DF80330013A5B008DF80330A7
:1042D0009DF90330002BF5D40A600A68032A2DD11A
:1042E0004FF4E06303EA02220A6001990170D0F8FA
:1042F000201941F47001C0F82019D0F8201941F0BC
:104300007041C0F82019FFF7F5FD4CF20800C2F229
:10431000010000210160FFF761FD4EF63470CEF21E
:104320000000016841F040410160FFF743FAFFF7E8
:1043300037FFFFF7CFFB002002B080BD4FF05000E9
:1043400080F31188BFF36F8FBFF34F8FFEE700003C
:1043500080B54FF0500080F31188BFF36F8FBFF32B
:104360004F8F00F063FB30B14EF60450CEF20000E8
:104370004FF080510160002080F3118880BD000063
:10438000B0B582B068B11D46ABB1F1B9EAB14FF03A
:10439000500080F31188BFF36F8FBFF34F8F00BFC2
:1043A000FEE74FF0500080F31188BFF36F8FBFF32B
:1043B0004F8F00BFFEE74FF0500080F31188BFF32E
:1043C0006F8FBFF34F8F00BFFEE751B14AB94FF077
:1043D000500080F31188BFF36F8FBFF34F8F00BF82
:1043E000FEE750230193019B502B0AD1069B019CB1
:1043F000012485F846400095FFF7E0F8284602B012
:10440000B0BD4FF0500080F31188BFF36F8FBFF342
:104410004F8F00BFFEE7000070B5F8B104460E46AE
:10442000FFF7E6FC2068D4E90F12002502FB010328
:10443000013901FB0201A563C4E90103FF20E1602A
:1044400084F8440084F8450004F110007EB1FFF7C1
:1044500089FC04F12400FFF785FC18E04FF05000C0
:1044600080F31188BFF36F8FBFF34F8FFEE70168B2
:1044700069B100F0CFFB50B14EF60450CEF200000F
:104480004FF080510160BFF34F8FBFF36F8FFFF785
:10449000D3FC012070BD00002DE9F04F83B00292E3
:1044A000B8B11D460E460446E9B1022D03D1E06BBA
:1044B000012840F09A8000F09FFA00BB0298F0B10A
:1044C0004FF0500080F31188BFF36F8FBFF34F8F11
:1044D000FEE74FF0500080F31188BFF36F8FBFF3FA
:1044E0004F8F00BFFEE7206C0028DED04FF0500059
:1044F00080F31188BFF36F8FBFF34F8FFEE7FFF795
:1045000077FCA06B022D58D0E16B884255D304F1A3
:10451000100801206F464FF0000B0DF108094FF015
:10452000805A00BF0299002900F07B80C00702D0AA
:104530003846FFF78BFDFFF77FFCFFF729FEFFF7FB
:1045400057FC94F84400FF2808BF84F844B094F85E
:104550004500FF2808BF84F845B0FFF76DFC3846DA
:10456000494600F095F900285ED12046FFF714F97E
:10457000A0B102994046FFF77FFD2046FFF7D0FA31
:1045800000F090FB78B94EF60450CEF20000C0F86F
:1045900000A0BFF34F8FBFF36F8F04E02046FFF7FB
:1045A000BFFA00F07FFBFFF723FCA06B022D04D0C5
:1045B000E16B88424FF00000B4D2204631462A46D3
:1045C000FEF740FF54F8241FC9B1204600F022FB3B
:1045D00008B34EF60450CEF200004FF08051016057
:1045E000BFF34F8FBFF36F8F15E04FF0500080F394
:1045F0001188BFF36F8FBFF34F8F00BFFEE750B13D
:104600004EF60450CEF200004FF080510160BFF32F
:104610004F8FBFF36F8FFFF70FFC012003B0BDE892
:10462000F08FFFF709FC04E02046FFF779FA00F06D
:1046300039FB002003B0BDE8F08F00002DE9F04306
:1046400081B0E8B11E46914605460F4609B3022ED9
:1046500002D1E86B012837D1FFF766FCEFF3118830
:104660004FF0500080F31188BFF36F8FBFF34F8F6F
:10467000A86B022E19D0E96B884216D300203FE0C8
:104680004FF0500080F31188BFF36F8FBFF34F8F4F
:10469000FEE7286C0028DAD04FF0500080F3118834
:1046A000BFF36F8FBFF34F8FFEE795F84540A86BC0
:1046B000284639463246FEF7C5FEFF2C0DD0601C59
:1046C00085F8450001201BE04FF0500080F3118871
:1046D000BFF36F8FBFF34F8FFEE755F8240F70B114
:1046E000284600F097FA0146B9F1000F4FF001009B
:1046F00006D000291CBF0120C9F8000000E00120FD
:1047000088F3118801B0BDE8F08300002DE9F04F77
:1047100085B0049298B10C460546002900F0A580AA
:1047200000F06AF9A8B9049898B14FF0500080F3EE
:104730001188BFF36F8FBFF34F8F00BFFEE74FF0BD
:10474000500080F31188BFF36F8FBFF34F8F00BF0E
:10475000FEE705F1240005F11009019002AF0DF10B
:10476000100A4FF000080AE02846FFF7D9F900F0D8
:1047700099FA2846FFF704F8002840F08480FFF7F4
:1047800037FBD5F838B0BBF1000F1DD028462146C5
:10479000FEF744FEABF10100A863286970B14846FA
:1047A00000F038FA50B14EF60450CEF200004FF04F
:1047B00080510160BFF34F8FBFF36F8FFFF73CFB5A
:1047C00000200126A0B95FE0049850B1B8F1000FB5
:1047D00002D13846FFF73AFC4FF00108012038B902
:1047E00052E0FFF729FB0026002000284CD000BF34
:1047F000FFF722FBFFF7CCFCFFF7FAFA95F844002D
:10480000FF2804BF002085F8440095F84500FF28E4
:1048100004BF002085F84500FFF70EFB38465146DF
:1048200000F036F800289FD12846FEF7A9FFB0B166
:1048300004990198FFF720FC2846FFF771F900F072
:1048400031FA00289BD14EF60450CEF200004FF012
:1048500080510160BFF34F8FBFF36F8F8FE7284602
:10486000FFF75EF900F01EFA89E7286C00283FF494
:1048700057AF4FF0500080F31188BFF36F8FBFF335
:104880004F8F00BFFEE70026304605B0BDE8F08F31
:10489000B0B5D0B10D4611B30446FFF7A9FA49F6F9
:1048A0000840C2F2010001682868421C21D049F684
:1048B000E8336268C2F20103D3F800C091421AD310
:1048C00023689C4517D0012422E04FF0500080F36C
:1048D0001188BFF36F8FBFF34F8F00BFFEE74FF01C
:1048E000500080F31188BFF36F8FBFF34F8F00BF6D
:1048F000FEE700240CE0891A884206D9401A286095
:104900002046FFF7A3FB002402E0002001242860DA
:10491000FFF792FA2046B0BD2DE9F04383B0074679
:104920009000984615468946FFF734F978B1064657
:104930005C20FFF72FF938B10446066354B94FF0F5
:10494000FF3003B0BDE8F0833046FFF78DFA002456
:10495000002CF4D0DDE90A10002284F85920CDE9BA
:104960000010384649462A4643460294FEF736FE72
:104970002046FEF797FC012003B0BDE8F08300005D
:1049800070B586B00B9CCCB10C9E06B35C2504952B
:10499000049D5C2D25D1049DDDF828C0022586F8F4
:1049A000595005AD3463CDE900C50296FEF716FEF9
:1049B0003046FEF777FC059806B070BD4FF050000A
:1049C00080F31188BFF36F8FBFF34F8FFEE74FF077
:1049D000500080F31188BFF36F8FBFF34F8F00BF7C
:1049E000FEE74FF0500080F31188BFF36F8FBFF3E5
:1049F0004F8F00BFFEE7000049F60440C2F20100FD
:104A00000068002804BF012070474CF6FC00C2F289
:104A100001000068B0FA80F04009400070470000D3
:104A200049F60840C2F20100006870472DE9F04FD6
:104A300081B04CF6FC00C2F20100006840B14CF6B7
:104A40009870C2F20100016800240131016092E017
:104A500049F60840C2F2010001684E1C066021D3ED
:104A60004CF29040C2F201000168096849B14FF070
:104A7000500080F31188BFF36F8FBFF34F8F00BFDB
:104A8000FEE740F2A812C2F2000201681368036058
:104A900049F6E8301160C2F201000168013101609D
:104AA000FEF7A6FF4CF69071C2F20101086840F2D1
:104AB000A41A4CF298488642C2F2000AC2F20108D7
:104AC00001D2002445E04CF29047C2F20107386859
:104AD0000024006898B34CF6041BC2F2010B19E0E5
:104AE000D9F82C00DBF80010884288BFCBF8000012
:104AF00000EB800008EB80002946FFF761F9D9F848
:104B00002C00DAF80010C96A3A68884228BF0124EC
:104B10001068B8B13868C068D0F80C904D4655F8A8
:104B2000040F864210D32846FFF7EEF8D9F8280084
:104B30000028D5D009F11800FFF7E6F8D0E74FF0CC
:104B4000FF3005E04FF0FF304CF69071C2F20101EA
:104B50000860DAF80000C06A00EB800058F8200016
:104B6000012849F61040C2F2010088BF0124006804
:104B7000002818BF0124204601B0BDE8F08F0000D6
:104B8000B0B580B1044640F2A410C2F20000006843
:104B9000A0420AD04FF0500080F31188BFF36F8F0E
:104BA000BFF34F8FFEE70020B0BD206D38B3013852
:104BB00020654FF0000018BFB0BDE16AE26C914281
:104BC0001CD0251D2846FFF79FF8E06CC0F1380186
:104BD000A1614CF60411E062C2F201010A68904240
:104BE00088BF08604CF2984100EB8000C2F20101DE
:104BF00001EB80002946FFF7E3F80120B0BD4FF03C
:104C0000500080F31188BFF36F8FBFF34F8F00BF49
:104C1000FEE70000B0B5C068C5687DB105F11804B5
:104C20002046FFF771F84CF6FC00C2F20100006864
:104C300068B149F6F030C2F201001DE04FF05000BB
:104C400080F31188BFF36F8FBFF34F8FFEE72C1DEA
:104C50002046FFF759F84CF60411C2F20101E86A48
:104C60000A68904288BF08604CF2984100EB8000CF
:104C7000C2F2010101EB80002146FFF7A1F840F2EA
:104C8000A411C2F20001E86A0968C96A884291BFAA
:104C9000002049F61041C2F20101012088BF0860DE
:104CA000B0BD00002DE9F04F81B04CF6FC04C2F21B
:104CB0000104206868B1FFF79BF820680138206084
:104CC000206880B10024FFF7B7F8204601B0BDE8A6
:104CD000F08F4FF0500080F31188BFF36F8FBFF358
:104CE0004F8F00BFFEE74CF6F800C2F201000068EB
:104CF00000285DD049F6F036C2F20106306849F668
:104D00001048C2F2010890B34CF604174CF29849CF
:104D100040F2A41BC2F20107C2F20109C2F2000B69
:104D20004FF0010AF068C56805F11800FEF7ECFFC6
:104D30002C1D2046FEF7E8FFE86A3968884288BFE4
:104D4000386000EB800009EB80002146FFF738F85F
:104D5000E86ADBF80010C96A884228BFC8F800A0DA
:104D600030680028DED1002D18BFFEF741FE4CF65A
:104D70009874C2F20104256855B10126FFF756FE6A
:104D8000002818BFC8F80060013DF7D1002020605E
:104D9000D8F8000070B14EF60450CEF200004FF08B
:104DA00080510160BFF34F8F0124BFF36F8F8AE7FB
:104DB000002488E7002486E780B586B0FEF7C8FAAD
:104DC0004DF20C00C2F20100006808B30020CDE9EA
:104DD000040005A804A903AAFEF7B6FFDDE9032035
:104DE0000221DDF814C0CDE9001043F60930C0F609
:104DF00000000CA10023CDF808C0FFF7C1FD49F663
:104E00000C41C2F20101086010B1012006B080BD62
:104E10004FF0500080F31188BFF36F8FBFF34F8FB7
:104E2000FEE700BF546D72205376630010B584B066
:104E3000A8B14DF20C04C2F2010484462068C0B14E
:104E40000529CDE90012CDF808C015DCFFF7D4FD27
:104E500001462068022916D1069A694615E04FF0EE
:104E6000500080F31188BFF36F8FBFF34F8F00BFE7
:104E7000FEE7002004B010BD69461A460023FFF784
:104E8000DDFB04B010BD694600220023FFF704FBE0
:104E900004B010BDF1EE100A4FF6FF71C0F2C03140
:104EA00020EA010040F04070E1EE100A7047000077
:104EB00000000000000001020304060708090000CA
:104EC0000000010203040000EC4E00080000000096
:104ED00000000000000000000000000000020000D0
:104EE000180000000000000000000000646566611A
:104EF000756C745461736B00384F0008000000201B
:104F000004000000C4010008404F000800C0012058
:104F100010000000C40100083C4F000804000020FD
:104F2000109C0100E0010008504F000810C0012053
:104F3000001C0000E001000801000000000000006B
:104F40000024F40010000000AAAAAAAA0000000091
:040000050800018965
:00000001FF
